:1000000012C02CC02BC02AC029C028C027C026C0BF
:1000100025C03EC2D1C246C121C020C024C81EC0D6
:100020001DC01CC01BC011241FBECFE5D4E0DEBF25
:10003000CDBF10E0A0E6B0E0EEECF5E102C0059027
:100040000D92A03DB107D9F711E0A0EDB0E001C0DD
:100050001D92AD35B107E1F715D0B7CAD1CFDF9307
:10006000CF93CDB7DEB7E1E3F0E082E88083E7E34A
:10007000F0E080E18083E8E3F0E088E28083CF91E4
:10008000DF910895DF93CF93CDB7DEB7E8DFF1D1ED
:1000900071D0DBD769D280E090E039D090932B010A
:1000A00080932A01A2E3B0E0E2E3F0E0808180687F
:1000B0008C937894EED085E580931B0185E4809342
:1000C0001C0185E690E090931F0180931E018EEF46
:1000D00090E0909321018093200151D280932901D7
:1000E0008091D100813029F41092D10080E090E01D
:1000F00024D88091D200813011F41092D2008091E6
:10010000DA00813051F71092DA0091D2E6CFDF9316
:10011000CF9300D0CDB7DEB79A83898389819A8146
:1001200029E930E0B90182D90F900F90CF91DF918A
:100130000895DF93CF9300D00F92CDB7DEB79B83A6
:100140008A83ECE3F0E08081882F90E082709070E9
:100150000097B9F7EEE3F0E08A819B819183808379
:10016000E09A8DB3898389810F900F900F90CF9182
:10017000DF910895DF93CF93CDB7DEB7E9E2F0E0EA
:1001800080E18083E0E4F0E01082A8E3B0E0E8E3FF
:10019000F0E0808181608C93EAE2F0E088E980837E
:1001A000E0E4F0E086E88083EBE2F0E082EC80833C
:1001B000CF91DF910895DF93CF930F92CDB7DEB744
:1001C0008983EBE2F0E08081882F90E0807290706C
:1001D0000097B9F3ECE2F0E0898180830F90CF9132
:1001E000DF910895DF93CF9300D000D0CDB7DEB775
:1001F0009B838A836C838C81882399F019820DC03C
:100200008981282F30E08A819B81FC01E20FF31F56
:100210008081D1DF89818F5F898399818C81891762
:1002200078F70F900F900F900F90CF91DF91089576
:10023000DF93CF9300D000D00F92CDB7DEB79D8370
:100240008C838C819D81E9D89A8389831B820FC01E
:100250008B81282F332727FD30958C819D81FC01D0
:10026000E20FF31F8081A7DF8B818F5F8B838B81F0
:10027000282F332727FD309589819A812817390740
:1002800038F30F900F900F900F900F90CF91DF9158
:100290000895DF93CF93CDB7DEB78EE38CDFCF9198
:1002A000DF9108951F920F920FB60F9211242F9392
:1002B0003F934F935F936F937F938F939F93AF93EE
:1002C000BF93EF93FF93DF93CF9300D000D00F92B3
:1002D000CDB7DEB7ECE2F0E0808180933B01809106
:1002E0003B0169DF80913B018D3079F030915A01FB
:1002F000832F90E020913B01FC01EB51FF4F2083C5
:10030000832F8F5F80935A019CC080915A01882F60
:1003100090E020913B01FC01EB51FF4F20831A82BA
:1003200019821092D7001092D8001092D9001B8227
:100330007DC08A81282F30E03D832C838C819D8174
:100340008130910569F12C813D812230310509F41C
:1003500049C08C819D81009709F065C08B81882FF1
:1003600090E0FC01EB51FF4F80818032A9F0898140
:10037000282F30E08B81882F90E0FC01EB51FF4F5C
:100380008081F901E05BFE4F808389818093D700F3
:1003900089818F5F898347C081E08A83198243C046
:1003A0008B81882F90E0FC01EB51FF4F80818032E0
:1003B000A9F08981282F30E08B81882F90E0FC0103
:1003C000EB51FF4F8081F901EA5BFE4F8083898109
:1003D0008093D80089818F5F898325C082E08A83DA
:1003E000198221C08B81882F90E0FC01EB51FF4FD7
:1003F00080818032A9F08981282F30E08B81882F7D
:1004000090E0FC01EB51FF4F8081F901E45CFE4F6D
:10041000808389818093D90089818F5F898303C01C
:1004200083E08A8319828B818F5F8B8390915A013D
:100430008B81981708F07DCF81E08093DA001092CD
:100440005A010F900F900F900F900F90CF91DF9166
:10045000FF91EF91BF91AF919F918F917F916F919C
:100460005F914F913F912F910F900FBE0F901F9072
:100470001895DF93CF93CDB7DEB7E3E5F0E082E0E8
:100480008083E9E5F0E081E08083CF91DF910895FA
:100490001F920F920FB60F9211248F93DF93CF9379
:1004A00000D0CDB7DEB78091DE008A8319828A81C1
:1004B000843011F481E089838A818F5F8093DE002C
:1004C0008981882329F081E08093D5001092DE0095
:1004D00080912C018F5F80932C0180912C018732B9
:1004E000C9F581E08093D30010922C018091DD004A
:1004F0008F5F8093DD008091DD00853029F41092BC
:10050000DD0081E08093D4008091DB008F5F8093D9
:10051000DB008091DB00843641F41092DB0081E047
:100520008093D00081E08093D2008091DB00823301
:1005300019F481E08093D2008091DC008F5F80937A
:10054000DC008091DC008A3029F41092DC0081E02C
:100550008093D1000F900F90CF91DF918F910F90EA
:100560000FBE0F901F901895DF93CF93CDB7DEB7D6
:10057000EDE2F0E080EC8083CF91DF910895DF938E
:10058000CF930F92CDB7DEB7E6E3F0E08081882FFE
:1005900090E084709070009749F08091DF0088238C
:1005A00011F01092DF0081E0898301C019828981F6
:1005B0000F90CF91DF9108951F920F920FB60F9277
:1005C00011242F933F934F938F939F93AF93BF9398
:1005D000EF93FF93DF93CF930F92CDB7DEB7AFE2E8
:1005E000B0E020916000309161004091DF00842FE5
:1005F00090E0F901E80FF91F80818C93842F8F5FC1
:100600008093DF00EFE2F0E0808189830F90CF914B
:10061000DF91FF91EF91BF91AF919F918F914F919A
:100620003F912F910F900FBE0F901F901895DF9361
:10063000CF93CDB7DEB7C55CD0400FB6F894DEBF20
:100640000FBECDBF9E01255F3F4FCD55DF4F398394
:100650002883C35AD04082E690E0CB55DF4F998380
:100660008883C55AD04098E0C955DF4F9883C75A50
:10067000D040CB55DF4FE881F981C55AD04000808A
:10068000CB55DF4F28813981C55AD0402F5F3F4F6E
:10069000CB55DF4F39832883C55AD040CD55DF4F26
:1006A000E881F981C35AD0400082CD55DF4F2881BF
:1006B0003981C35AD0402F5F3F4FCD55DF4F39832B
:1006C0002883C35AD040C955DF4F3881C75AD0401C
:1006D0003150C955DF4F3883C75AD040C955DF4F15
:1006E0008881C75AD040882321F6FE017396C855E9
:1006F000DF4FF983E883C85AD0402AE630E0C65578
:10070000DF4F39832883CA5AD0403FE0C455DF4FBA
:100710003883CC5AD040C655DF4FE881F981CA5A98
:10072000D0400080C655DF4F28813981CA5AD04059
:100730002F5F3F4FC655DF4F39832883CA5AD040B9
:10074000C855DF4FE881F981C85AD0400082C855AA
:10075000DF4F28813981C85AD0402F5F3F4FC8559D
:10076000DF4F39832883C85AD040C455DF4F3881C2
:10077000CC5AD0403150C455DF4F3883CC5AD0408A
:10078000C455DF4F8881CC5AD040882321F6FE0122
:10079000B296C355DF4FF983E883CD5AD04029E79D
:1007A00030E0C155DF4F39832883CF5AD0403DE038
:1007B000CF54DF4F3883C15BD040C155DF4FE88154
:1007C000F981CF5AD0400080C155DF4F288139814F
:1007D000CF5AD0402F5F3F4FC155DF4F3983288319
:1007E000CF5AD040C355DF4FE881F981CD5AD04070
:1007F0000082C355DF4F28813981CD5AD0402F5F09
:100800003F4FC355DF4F39832883CD5AD040CF5453
:10081000DF4F3881C15BD0403150CF54DF4F388338
:10082000C15BD040CF54DF4F8881C15BD04088236B
:1008300021F6FE01BF96CE54DF4FF983E883C25BF9
:10084000D04026E830E0CC54DF4F39832883C45BA6
:10085000D04038E0CA54DF4F3883C65BD040CC5418
:10086000DF4FE881F981C45BD0400080CC54DF4F7A
:1008700028813981C45BD0402F5F3F4FCC54DF4F7C
:1008800039832883C45BD040CE54DF4FE881F9819F
:10089000C25BD0400082CE54DF4F28813981C25BD9
:1008A000D0402F5F3F4FCE54DF4F39832883C25B48
:1008B000D040CA54DF4F3881C65BD0403150CA5453
:1008C000DF4F3883C65BD040CA54DF4F8881C65B98
:1008D000D040882321F6FE01F796C954DF4FF983F3
:1008E000E883C75BD0402EE830E0C754DF4F398340
:1008F0002883C95BD0403DE0C554DF4F3883CB5BD4
:10090000D040C754DF4FE881F981C95BD0400080F7
:10091000C754DF4F28813981C95BD0402F5F3F4FDB
:10092000C754DF4F39832883C95BD040C954DF4F98
:10093000E881F981C75BD0400082C954DF4F28812C
:100940003981C75BD0402F5F3F4FC954DF4F398398
:100950002883C75BD040C554DF4F3881CB5BD04084
:100960003150C554DF4F3883CB5BD040C554DF4F87
:100970008881CB5BD040882321F6CE018C5B9F4FD2
:10098000C454DF4F99838883CC5BD040EBE9F0E01F
:10099000C254DF4FF983E883CE5BD040F4E1C0540A
:1009A000DF4FF883C05CD040C254DF4FE881F9814B
:1009B000CE5BD0400080C254DF4F28813981CE5BAE
:1009C000D0402F5F3F4FC254DF4F39832883CE5B27
:1009D000D040C454DF4FE881F981CC5BD040008225
:1009E000C454DF4F28813981CC5BD0402F5F3F4F0B
:1009F000C454DF4F39832883CC5BD040C054DF4FD1
:100A00003881C05CD0403150C054DF4F3883C05C67
:100A1000D040C054DF4F8881C05CD040882321F68D
:100A2000CE01885A9F4FCF53DF4F99838883C15C93
:100A3000D040EFEAF0E0CD53DF4FF983E883C35CA9
:100A4000D040F7E1CB53DF4FF883C55CD040CD53A6
:100A5000DF4FE881F981C35CD0400080CD53DF4F88
:100A600028813981C35CD0402F5F3F4FCD53DF4F8A
:100A700039832883C35CD040CF53DF4FE881F981AD
:100A8000C15CD0400082CF53DF4F28813981C15CE7
:100A9000D0402F5F3F4FCF53DF4F39832883C15C56
:100AA000D040CB53DF4F3881C55CD0403150CB5361
:100AB000DF4F3883C55CD040CB53DF4F8881C55CA6
:100AC000D040882321F680915001CE55DF4F188207
:100AD000C25AD040883631F491E0CE55DF4F98832A
:100AE000C25AD04080915101CF55DF4F1882C15A70
:100AF000D040853631F4E1E0CF55DF4FE883C15A6D
:100B0000D040CE55DF4F8881C25AD040CF55DF4FFD
:100B1000F881C15AD0408F23282F30E0C156DF4FD3
:100B200039832883CF59D04080915201C356DF4F7B
:100B300019821882CD59D0408C3641F481E090E082
:100B4000C356DF4F99838883CD59D040C156DF4FBC
:100B5000E881F981CF59D040C356DF4F28813981D0
:100B6000CD59D040E223F323C556DF4FF983E88304
:100B7000CB59D04080915301C756DF4F198218825C
:100B8000C959D040803741F481E090E0C756DF4F2B
:100B900099838883C959D040C556DF4F8881998190
:100BA000CB59D040C756DF4FE881F981C959D040B1
:100BB0008E239F23009799F0CE010B9639DBCE014F
:100BC000439636DBCE01829633DBCE018F9630DB47
:100BD000CE01C7962DDBCE018C5B9F4F29DB809128
:100BE0005001C856DF4F1882C859D040833731F4BE
:100BF000F1E0C856DF4FF883C859D04080915101C9
:100C0000C956DF4F1882C759D040883631F421E0E9
:100C1000C956DF4F2883C759D040C856DF4F888157
:100C2000C859D040C956DF4F3881C759D0408323B7
:100C3000E82FF0E0CB56DF4FF983E883C559D04069
:100C400080915201CD56DF4F19821882C359D0408E
:100C50008F3641F421E030E0CD56DF4F39832883D1
:100C6000C359D040CB56DF4F88819981C559D040B8
:100C7000CD56DF4FE881F981C359D0408E239F23A1
:100C8000CF56DF4F99838883C159D040809153015B
:100C9000C157DF4F19821882CF58D040873741F4AF
:100CA00021E030E0C157DF4F39832883CF58D0404F
:100CB000CF56DF4F88819981C159D040C157DF4F4E
:100CC000E881F981CF58D0408E239F23009709F403
:100CD0005DC080914601C257DF4F1882CE58D04088
:100CE000863731F4F1E0C257DF4FF883CE58D04059
:100CF00080914701C357DF4F1882CD58D0408536C9
:100D000031F421E0C357DF4F2883CD58D040C2577C
:100D1000DF4F8881CE58D040C357DF4F3881CD5840
:100D2000D0408323882321F0CE01885A9F4F80DA58
:100D300080914601C457DF4F1882CC58D04083378A
:100D400031F481E0C457DF4F8883CC58D040809184
:100D50004701C557DF4F1882CB58D040843731F454
:100D600091E0C557DF4F9883CB58D040C457DF4F31
:100D70008881CC58D040C557DF4FE881CB58D04050
:100D80008E23882319F081E08093D6008091500152
:100D9000C657DF4F1882CA58D040833731F4F1E08C
:100DA000C657DF4FF883CA58D04080915101C757CA
:100DB000DF4F1882C958D040843731F421E0C7573B
:100DC000DF4F2883C958D040C657DF4F8881CA58A3
:100DD000D040C757DF4F3881C958D0408323E82F10
:100DE000F0E0C957DF4FF983E883C758D0408091BE
:100DF0005201CB57DF4F19821882C558D0408F3629
:100E000041F421E030E0CB57DF4F39832883C558C8
:100E1000D040C957DF4F88819981C758D040CB5700
:100E2000DF4FE881F981C558D0408E239F23CD57ED
:100E3000DF4F99838883C358D04080915301CF57A7
:100E4000DF4F19821882C158D040803741F421E029
:100E500030E0CF57DF4F39832883C158D040CD577A
:100E6000DF4F88819981C358D040CF57DF4FE88149
:100E7000F981C158D0408E239F23009711F0109222
:100E8000D60080915001C058DF4F1882C058D04022
:100E9000833731F4F1E0C058DF4FF883C058D040B9
:100EA00080915101C158DF4F1882CF57D04085360D
:100EB00031F421E0C158DF4F2883CF57D040C058CC
:100EC000DF4F8881C058D040C158DF4F3881CF579D
:100ED000D0408323E82FF0E0EF96FFAFEEAFEF971F
:100EE00080915201ED961FAE1EAEED97843731F41E
:100EF00021E030E0ED963FAF2EAFED97EF968EAD4F
:100F00009FADEF97ED96EEADFFADED978E239F234E
:100F1000009739F180914601EB961FAEEB9783362F
:100F200021F4F1E0EB96FFAFEB9780914701EA9651
:100F30001FAEEA978A3721F421E0EA962FAFEA97AD
:100F4000EB968FADEB97EA963FADEA978323882324
:100F500041F08CE391E044D290932B0180932A01DD
:100F6000F0D180915001E9961FAEE997823721F4C4
:100F700081E0E9968FAFE99780915101E8961FAE25
:100F8000E897853621F491E0E8969FAFE897E996D7
:100F90008FADE997E896EFADE8978E23282F30E0E4
:100FA000E7963FAF2EAFE79780915201E5961FAECF
:100FB0001EAEE597833731F481E090E0E5969FAF70
:100FC0008EAFE597E796EEADFFADE797E5962EADD0
:100FD0003FADE597E223F323E396FFAFEEAFE39750
:100FE00080915301E1961FAE1EAEE197853631F434
:100FF00081E090E0E1969FAF8EAFE197E3968EADF2
:101000009FADE397E196EEADFFADE1978E239F2371
:10101000009709F00BD03DD9CB53DF4F0FB6F894B2
:10102000DEBF0FBECDBFCF91DF910895DF93CF9389
:10103000CDB7DEB7F89488E190E028E00FB6F894D9
:10104000A89581BD0FBE21BDFFCFDF93CF93CDB754
:10105000DEB7E7E2F0E01082E6E2F0E08FE88083BE
:10106000CF91DF9108951F920F920FB60F92112426
:101070002F933F934F935F938F939F93EF93FF93A0
:10108000DF93CF93CDB7DEB7E6E2F0E01082809138
:10109000C600482F50E0E4E2F0E0808191819C019D
:1010A000CA01880F991FFC01E35DFE4F3183208345
:1010B0008091C600482F50E0882F90E0880F991F3C
:1010C000FC01E35DFE4F2081318180912A019091E6
:1010D0002B01281B390BCA01880F991FFC01E35D06
:1010E000FE4F318320838091C600882F90E0880FC7
:1010F000991FFC01E35DFE4F8081918199235CF48F
:101100008091C600882F90E0880F991FFC01E35D55
:10111000FE4F1182108281E08093E000CF91DF9139
:10112000FF91EF919F918F915F914F913F912F91FF
:101130000F900FBE0F901F901895DF93CF93CDB7F0
:10114000DEB76C970FB6F894DEBF0FBECDBF8C8FA5
:101150008091C6008F5F8093C6008091C600853065
:1011600008F4DFC01092C6001F82188619861A86FE
:101170001B8628C08B85882F90E0880F991FFC0163
:10118000E35DFE4F2081318189E790E0AC01249F2F
:10119000C001259F900D349F900D11249C01442780
:1011A00037FD4095542F8F819885A985BA85820F88
:1011B000931FA41FB51F8F839887A987BA878B8534
:1011C0008F5F8B878B858530A8F28F819885A98565
:1011D000BA8525E030E040E050E0BC01CD01BFD150
:1011E000DA01C9018B839C83AD83BE832091E1002A
:1011F0003091E2004091E3005091E4008F819885A6
:10120000A985BA85820F931FA41FB51F8093E100A3
:101210009093E200A093E300B093E4008091E1009A
:101220009091E200A091E300B091E40020EA3CE854
:1012300040E050E0BC01CD0192D1DA01C9019A83AE
:1012400089839DD98823E9F385E580931B018B81F0
:101250009C81AD81BE8128EE33E040E050E0BC01CE
:10126000CD017DD1DA01C90180931C018B819C8164
:10127000AD81BE8128EE33E040E050E0BC01CD01FD
:101280006ED1DC01CB0124E630E040E050E0BC014F
:10129000CD0165D1DA01C90180931D0185E690E099
:1012A00090931F0180931E0189819A81909321015F
:1012B000809320018091D600813099F580912D0195
:1012C00090912E019E01245F3F4FB9014AE050E00A
:1012D00022D1CE010C96ACD787EC90E0A9D78B81B8
:1012E0009C81AD81BE819E01245F3F4FBC01CD0139
:1012F000A9012AE030E0ECD0CE010C9699D787EC1A
:1013000090E096D789819A819E01245F3F4FB90171
:101310004AE050E0B6D0CE010C968AD78CEC90E033
:1013200087D7E7E2F0E01082E6E2F0E08FEC80831E
:101330006C960FB6F894DEBF0FBECDBFCF91DF9194
:101340000895DF93CF93CDB7DEB780E090E0209192
:101350002A0130912B01B90103D0CF91DF9108957B
:10136000DF93CF9300D000D0CDB7DEB79A838983C7
:101370007C836B8389819A812B813C8149EC59E084
:10138000B9016AD00F900F900F900F90CF91DF911D
:101390000895DF93CF9300D00F92CDB7DEB79A8335
:1013A00089836B83ECE3F0E08081882F90E082708A
:1013B00090700097B9F7EEE3F0E089819A8191830C
:1013C0008083EDE3F0E08B8180830FB6F894E29A9E
:1013D000E19A0FBE0F900F900F90CF91DF9108957B
:1013E000FC0188279927E89421912032E9F32930DC
:1013F00010F02E30C8F32B3239F02D3231F46894CE
:1014000003C05ED0820F911D219120532A30C8F372
:101410001EF4909581959F4F0895FC010190002046
:10142000E9F7809590958E0F9F1F0895DF92EF92B8
:10143000FF920F931F937B018C01FB010995D82E1E
:10144000C8010196F7010995982F8D2D1F910F91D5
:10145000FF90EF90DF900895DF92EF92FF920F934D
:101460001F93D72E7A018C01FA010995C8010196C4
:101470006D2DF70109951F910F91FF90EF90DF906F
:101480000895FB019F01E8944230BCF04532ACF472
:101490004A3029F497FB1EF4909581959F4F642F55
:1014A00077277FD0805D8A330CF0895D8193CB01F3
:1014B0000097A9F716F45DE251931082C9013FC06D
:1014C0007AE0979F902D879F802D910D112408958C
:1014D000FA01CF93FF93EF932230C4F02532B4F496
:1014E000C22F2C2F332744275527FF93EF9337D054
:1014F000EF91FF91605D6A330CF0695D6193B90112
:10150000CA01605070408040904059F710828F911E
:101510009F91CF9114C0FB019F0142306CF0453286
:101520005CF4642F77273DD0805D8A330CF0895DB1
:101530008193CB010097A9F71082C90100C0DC019B
:10154000FC01672F71917723E1F7329704C07C91FA
:101550006D9370836291AE17BF07C8F30895A1E23F
:101560001A2EAA1BBB1BFD010DC0AA1FBB1FEE1F1D
:10157000FF1FA217B307E407F50720F0A21BB30B68
:10158000E40BF50B661F771F881F991F1A9469F7E4
:1015900060957095809590959B01AC01BD01CF0140
:1015A0000895AA1BBB1B51E107C0AA1FBB1FA617AA
:1015B000B70710F0A61BB70B881F991F5A95A9F7FC
:0E15C00080959095BC01CD010895F894FFCF61
:1015CE001B0168656C70200D000073686F772076C4
:1015DE00657273696F6E0D000073686F77206572A8
:1015EE00726F720D000072657365740D0000736882
:1015FE006F77207374726F6D0D00007365742063C6
:10160E007A202863616C5F7A65726F290D00004540
:10161E0050492D5374726F6D205665722E3A2030DC
:10162E002E302E310D000520202000000D00000070
:00000001FF
